:100000009BC41895189518951895189518951895D6
:100010001895B7CE189518951895189518951895A0
:1000200018951895189500E0302E0FEF502E702E71
:1000300000EC402E0FEF602E802E00E0902E0FEF90
:10004000B02ED02E00E8A02E0FEBC02E0FEFE02E2A
:10005000C8DBC7DBC6DBC5DBC4DBC3DBC2DBC1DBA4
:10006000C0DB00E0302E502E0FEF702E00EC402E43
:10007000602E0FEF802E00E0902EB02E0FEFD02ECE
:1000800000ECA02E00E8C02E0FEFE02EAADBA9DBCB
:10009000A8DBA7DBA6DBA5DBA4DBA3DBA2DB0FEFE2
:1000A000302E00E0502E0FEF702E402E00EC602E10
:1000B0000FEF802E902E00E0B02E0FEFD02EA02E4E
:1000C00000E8C02E0FEBE02E8CDB8BDB8ADB89DBBC
:1000D00088DB87DB86DB85DB84DB0FEF302E00E0FF
:1000E000502E702E0FEF402E00EC602E802E0FEF62
:1000F000902E00E0B02ED02E0FEFA02E00ECC02EE0
:1001000000E8E02E6EDB6DDB6CDB6BDB6ADB69DB52
:1001100068DB67DB66DB0FEF302E502E00E0702EC1
:100120000FEF402E602E00EC802E0FEF902EB02EA1
:1001300000E0D02E0FEBA02E0FEFC02E00E8E02E37
:1001400050DB4FDB4EDB4DDB4CDB4BDB4ADB49DB73
:1001500048DB00E0302E0FEF502E00E0702E00EC58
:10016000402E0FEF602E00EC802E00E0902E0FEF5F
:10017000B02E00E0D02E00E8A02E0FEBC02E00E83D
:10018000E02E2FDB2EDB2DDB2CDB2BDB2ADB29DB30
:1001900028DB27DB00E0302E502E702E00EC402EA6
:1001A000602E802E00E0902EB02ED02E00E8A02EE3
:1001B00000ECC02EE02E15DB14DB13DB12DB11DBB1
:1001C00010DB0FDB0EDB0DDB089505E3302E08E5B9
:1001D000502E09EA702E05EF402E08ED602E09EE34
:1001E000802E04ED902E01E6B02E06EAD02E04E912
:1001F000A02E01EEC02E06EEE02EF3DAF2DAF1DAEE
:10020000F0DAEFDAEEDAEDDAECDAEBDA03EA302EF6
:1002100005E1502E0AE3702E03EE402E05ED602E10
:100220000AEF802E0EE8902E04E5B02E08EED02EB8
:100230000EE8A02E04EDC02E08EEE02ED2DAD1DAC0
:10024000D0DACFDACEDACDDACCDACBDACADA0AE62D
:10025000302E01EA502E03E5702E0AEE402E01EEFC
:10026000602E03ED802E09EA902E06E8B02E0DE4F4
:10027000D02E09EAA02E06ECC02E0DECE02EB1DA4D
:10028000B0DAAFDAAEDAADDAACDAABDAAADAA9DA3A
:1002900006E5302E0AE2502E05E6702E06ED402EC1
:1002A0000AEE602E05EE802E09E5902E08EAB02EAB
:1002B00005E9D02E09E9A02E08EEC02E05EDE02EAE
:1002C00090DA8FDA8EDA8DDA8CDA8BDA8ADA89DAFA
:1002D00088DA05EC302E02E5502E06EA702E05EC89
:1002E000402E02ED602E06EE802E07E1902E09E4EE
:1002F000B02E0AE9D02E07E9A02E09ECC02E0AED97
:10030000E02E6FDA6EDA6DDA6CDA6BDA6ADA69DAF5
:1003100068DA67DA0CEA302E05E4502E0AEC702E0B
:100320000CEE402E05EC602E0AEC802E02EB902E97
:1003300005E1B02E0BE2D02E02EBA02E05EDC02E73
:100340000BEEE02E4EDA4DDA4CDA4BDA4ADA49DAC5
:1003500048DA47DA46DA0AE9302E04EA502E0CE58C
:10036000702E0AE9402E04EE602E0CED802E0AE677
:10037000902E02E9B02E01E7D02E0AEAA02E02ED5F
:10038000C02E01EFE02E2DDA2CDA2BDA2ADA29DA68
:1003900028DA27DA26DA25DA09E5302E0AE8502E9F
:1003A00005E9702E09ED402E0AEC602E05ED802E39
:1003B00005E6902E0AE2B02E06E5D02E05EAA02E24
:1003C0000AEEC02E06EDE02E0CDA0BDA0ADA09DAB4
:1003D00008DA07DA06DA05DA04DA08950FEF302EC4
:1003E0000FE0502E00EF702E0FEF402E00EC602E2D
:1003F0000FEF802E902E00E0B02E0FEFD02E03E8EE
:10040000A02E0CEFC02E0FEFE02EEBD9EAD9E9D9E0
:10041000E8D9E7D9E6D9E5D9E4D9E3D900EF302E18
:100420000FEF502E0FE0702E0FEF402E00EC602EDD
:100430000FEF802E902E00E0B02E0FEFD02E0FEB9E
:10044000A02E00ECC02E0FEFE02ECBD9CAD9C9D90F
:10045000C8D9C7D9C6D9C5D9C4D9C3D90FE0302E98
:1004600000EF502E0FEF702E402E0FEC602E00EF9D
:10047000802E0FEF902E00E0B02E0FEFD02E0FEB5E
:10048000A02E00ECC02E0FEFE02EABD9AAD9A9D92F
:10049000A8D9A7D9A6D9A5D9A4D9A3D90FEF302E09
:1004A00000E0502E0FEF702E00EF402E0FEF602E69
:1004B0000FEC802E0FEF902E03E0B02E0CEFD02E1D
:1004C0000FEBA02E00ECC02E0FEFE02E8AD989D9B9
:1004D00088D987D986D985D984D983D982D90FEF8C
:1004E000302E00E0502E0FEF702E0FEC402E00EF5C
:1004F000602E0FEF802E0CEF902E0FE3B02E03EC4A
:10050000D02E0FEBA02E00ECC02E0FEFE02E69D9FD
:1005100068D967D966D965D964D963D962D961D9EF
:100520000FEF302E00E0502E0FEF702E402E00EC1B
:10053000602E0FEF802E03EC902E0CEFB02E0FE309
:10054000D02E0FEBA02E03ECC02E0CEFE02E49D9DD
:1005500048D947D946D945D944D943D942D941D9AF
:100560000FEF302E00E0502E0FEF702E402E00ECDB
:10057000602E0FEF802E0FE3902E00ECB02E0FEFC9
:10058000D02E0CEBA02E0FEFC02E03ECE02E29D9BD
:1005900028D927D926D925D924D923D922D921D96F
:1005A000089507EF302E08E1502E0FEE702E07EF62
:1005B000402E08ED602E0FEE802E0FED902E00E6FF
:1005C000B02E0FEBD02E0FE9A02E00EEC02E0FEFB5
:1005D000E02E07D906D905D904D903D902D901D902
:1005E00000D9FFD80FEE302E01E1502E0EEF702E05
:1005F0000FEE402E01ED602E0EEF802E0FEB902EB1
:1006000004E4B02E0BEFD02E0FEBA02E04ECC02E86
:100610000BEFE02EE6D8E5D8E4D8E3D8E2D8E1D86D
:10062000E0D8DFD8DED80EEF302E01E2502E0FEDED
:10063000702E0EEF402E01EE602E0FED802E0BEF90
:10064000902E04E8B02E0FE7D02E0BEBA02E04EC7A
:10065000C02E0FEFE02EC5D8C4D8C3D8C2D8C1D899
:10066000C0D8BFD8BED8BDD80FED302E02E2502E74
:100670000DEF702E0FED402E02EE602E0DEF802E4E
:100680000FE7902E08E8B02E07EFD02E0FEBA02E2C
:1006900008ECC02E07EFE02EA4D8A3D8A2D8A1D88A
:1006A000A0D89FD89ED89DD89CD80DEF302E02E4BC
:1006B000502E0FEB702E0DEF402E02EC602E0FEF40
:1006C000802E07EF902E09E0B02E0EEFD02E07EB14
:1006D000A02E09ECC02E0EEFE02E83D882D881D850
:1006E00080D87FD87ED87DD87CD87BD80FEB302EB1
:1006F00004E4502E0BEF702E0FEF402E04EC602E12
:100700000BEF802E0EEF902E01E1B02E0FEED02ECB
:100710000EEBA02E01EDC02E0FEEE02E62D861D8B8
:1007200060D85FD85ED85DD85CD85BD85AD80BEF5C
:10073000302E04E8502E0FE7702E0BEF402E04EC05
:10074000602E0FEF802E0FEE902E02E1B02E0DEFF7
:10075000D02E0FEAA02E02EDC02E0DEFE02E41D8D4
:1007600040D83FD83ED83DD83CD83BD83AD839D8E5
:100770000FE7302E08E8502E07EF702E0FEF402EB7
:1007800008EC602E07EF802E0DEF902E02E2B02EC7
:100790000FEDD02E0DEBA02E02EEC02E0FEDE02EB1
:1007A00020D81FD81ED81DD81CD81BD81AD819D8A5
:1007B00018D808950FEF302E402E502E602E00E0F6
:1007C000702E00EC802E0FEF902EA02EB02E0FEB8F
:1007D000C02E00E0D02E00ECE02E03D802D801D8C5
:1007E00000D8FFD7FED7FDD7FCD7FBD700E0302ECF
:1007F00000EC402E0FEF502E602E702E802E00E069
:10080000902E00ECA02E0FEFB02EC02ED02E0FEBAE
:10081000E02EE7D7E6D7E5D7E4D7E3D7E2D7E1D7AD
:10082000E0D7DFD70FEF302E402E00E0502E00EC47
:10083000602E0FEF702E802E902E0FEBA02E00E07A
:10084000B02E00ECC02E0FEFD02EE02ECAD7C9D7A5
:10085000C8D7C7D7C6D7C5D7C4D7C3D7C2D70895B7
:10086000F39410E0211609F0FBCF3F2CF39411E034
:10087000211609F0FBCF1F2C5EDA412CF39415E012
:10088000211609F0FBCF9F2CF39411E0211609F0FB
:10089000FBCF1F2C50DAA12CF39413E0211609F0A2
:1008A000FBCF7F2CF39414E0211609F0FBCF1F2C13
:1008B00042DA812CF39410E0211609F0FBCFDF2CF3
:1008C000F39414E0211609F0FBCF1F2C34DAE12C4D
:1008D000F39415E0211609F0FBCF032C07201F2C01
:1008E0002FDA512CF39412E0211609F0FBCF042CDF
:1008F00008201F2C25DA1FDA612CF39413E021164F
:1009000009F0FBCF092C0D201F2C1ADAB12CF3941F
:1009100012E0211609F0FBCF0A2C0E201F2C10DA52
:100920000ADAC12C5ED75DD75CD75BD75AD759D7C7
:1009300058D757D756D708950FE50DBF04E00EBF1F
:1009400003E003BF01E009BF00E805BF789400E0C1
:1009500000936000009361000FE7002E07BA0FEFCD
:10096000002E08BA01BA02BA0FE3002E04BA05BA83
:1009700001E1009361008DDAF39410E0211609F093
:10098000FBCF3F2CF39411E0211609F0FBCF1F2C75
:10099000D2D9412CF39415E0211609F0FBCF9F2CFE
:1009A000F39411E0211609F0FBCF1F2CC4D9A12C20
:1009B000F39413E0211609F0FBCF7F2CF39414E09D
:1009C000211609F0FBCF1F2CB6D9812CF39410E02F
:1009D000211609F0FBCFDF2CF39414E0211609F067
:1009E000FBCF1F2CA8D9E12CF39415E0211609F0B8
:1009F000FBCF5F2CF39412E0211609F0FBCF1F2CE4
:100A00009AD9612CF39413E0211609F0FBCFBF2C87
:100A1000F39412E0211609F0FBCF1F2C8CD9C12CC6
:100A2000E0D60895F39410E0211609F0FBCF3F2C97
:100A3000F39411E0211609F0FBCF1F2C7CD9412C37
:100A4000F39415E0211609F0FBCF9F2CF39411E0ED
:100A5000211609F0FBCF1F2C6ED9A12CF39413E0C3
:100A6000211609F0FBCF7F2CF39414E0211609F036
:100A7000FBCF1F2C60D9812CF39410E0211609F0D4
:100A8000FBCFDF2CF39414E0211609F0FBCF1F2CD1
:100A900052D9E12CF39415E0211609F0FBCF032C79
:100AA00007201F2C4DD9512CF39412E0211609F088
:100AB000FBCF042C08201F2C43D93DD9612CF39483
:100AC00013E0211609F0FBCF092C0D201F2C38D97B
:100AD000B12CF39412E0211609F0FBCF0A2C0E2062
:100AE0001F2C2ED928D9C12C7CD608950FEF302E7B
:100AF000402E00E0502E00EC602E0FEF702E802E66
:100B0000902E0FEBA02E00E0B02E00ECC02E0FEFC9
:100B1000D02EE02E66D608950FEF302E402E502EA8
:100B2000602E00E0702E00EC802E0FEF902EA02E95
:100B3000B02E0FEBC02E00E0D02E00ECE02E51D6F0
:100B400000E0302E00EC402E0FEF502E602E702E65
:100B5000802E00E0902E00ECA02E0FEFB02EC02EC5
:100B6000D02E0FEBE02E3DD60FEF302E402E00E0C2
:100B7000502E00EC602E0FEF702E802E902E0FEB7B
:100B8000A02E00E0B02E00ECC02E0FEFD02EE02EF5
:100B900028D60895A4D3A3D3A2D3A1D3A0D3BCDFD6
:100BA000BBDFBADFB9DFB8DFB7DF25D224D223D26B
:100BB00022D221D220D2E8D2E7D2E6D2E5D2E4D2C4
:100BC000E3D2B6D0B5D0B4D0B3D0B2D0B1D079D111
:100BD00078D177D176D175D174D173D123D622D67D
:100BE00021D620D61FD61ED61DDF1CDF1BDF1ADF45
:100BF00019DF18DF17DF16DF15DF14DF13DF12DF51
:100C000011DF10DF0FDFD6DDD5DDD4DDD3DDD2DDA2
:100C1000D1DDC7DCC6DCC5DCC4DCC3DCC2DCDEDBAA
:100C2000DDDBDCDBDBDBDADBD9DBCFDACEDACDDA3E
:100C3000CCDACBDACADAF7D9F6D9F5D9F4D9F3D9BF
:100C4000F2D90EDE0DDE0CDE0BDE0ADE09DE08DE7A
:100C500007DE06DE05DE04DE03DE02DE01DE00DE88
:100C600008953DD33CD33BD33AD339D355DF54DF3A
:100C700053DF52DF51DF50DF9DDD9CDD9BDD9ADDD0
:100C800099DD98DDB8D1B7D1B6D1B5D1B4D1B3D152
:100C900088DC87DC86DC85DC84DC83DC75D274D27E
:100CA00073D272D271D270D299DB98DB97DB96DB6C
:100CB00095DB94DB3DD03CD03BD03AD039D038D016
:100CC00084DA83DA82DA81DA80DA7FDAFAD0F9D06C
:100CD000F8D0F7D0F6D0F5D0F4D0A5D9A4D9A3D9BF
:100CE000A2D9A1D9A0D99ED59DD59CD59BD59AD561
:100CF00099D598DE97DE96DE95DE94DE93DE92DE61
:100D000091DE90DE8FDE8EDE8DDE8CDE8BDE8ADE87
:100D1000A7DDA6DDA5DDA4DDA3DDA2DDA1DDA0DDCF
:100D20009FDD9EDD9DDD9CDD9BDD9ADD99DD0895D7
:100D300005E3302E08E5502E09EA702E05EF402E0F
:100D400008ED602E09EE802E04ED902E01E6B02E07
:100D500006EAD02E04E9A02E01EEC02E06EEE02E0B
:100D600040D503EA302E05E1502E0AE3702E03EE43
:100D7000402E05ED602E0AEF802E0EE8902E04E541
:100D8000B02E08EED02E0EE8A02E04EDC02E08EEF8
:100D9000E02E27D50AE6302E01EA502E03E5702E0C
:100DA0000AEE402E01EE602E03ED802E09EA902E11
:100DB00006E8B02E0DE4D02E09EAA02E06ECC02ED7
:100DC0000DECE02E0ED506E5302E0AE2502E05E69B
:100DD000702E06ED402E0AEE602E05EE802E09E5FF
:100DE000902E08EAB02E05E9D02E09E9A02E08EED3
:100DF000C02E05EDE02EF5D405EC302E02E5502E88
:100E000006EA702E05EC402E02ED602E06EE802ED6
:100E100007E1902E09E4B02E0AE9D02E07E9A02EB2
:100E200009ECC02E0AEDE02EDCD40CEA302E05E4ED
:100E3000502E0AEC702E0CEE402E05EC602E0AECC3
:100E4000802E02EB902E05E1B02E0BE2D02E02EBAD
:100E5000A02E05EDC02E0BEEE02EC3D40AE9302EF5
:100E600004EA502E0CE5702E0AE9402E04EE602EA6
:100E70000CED802E0AE6902E02E9B02E01E7D02E6E
:100E80000AEAA02E02EDC02E01EFE02EAAD409E559
:100E9000302E0AE8502E05E9702E09ED402E0AEC9E
:100EA000602E05ED802E05E6902E0AE2B02E06E5B6
:100EB000D02E05EAA02E0AEEC02E06EDE02E91D42B
:100EC000089500E0302E0FEF502E702E00EC402ED3
:100ED0000FEF602E802E00E0902E0FEFB02ED02E60
:100EE00000E8A02E0FEBC02E0FEFE02E7AD400E02A
:100EF000302E502E0FEF702E00EC402E602E0FEF94
:100F0000802E00E0902EB02E0FEFD02E00ECA02E01
:100F100000E8C02E0FEFE02E64D40FEF302E00E07B
:100F2000502E0FEF702E402E00EC602E0FEF802E13
:100F3000902E00E0B02E0FEFD02EA02E00E8C02E95
:100F40000FEBE02E4ED40FEF302E00E0502E702E1F
:100F50000FEF402E00EC602E802E0FEF902E00E061
:100F6000B02ED02E0FEFA02E00ECC02E00E8E02E09
:100F700038D40FEF302E502E00E0702E0FEF402EA1
:100F8000602E00EC802E0FEF902EB02E00E0D02EC1
:100F90000FEBA02E0FEFC02E00E8E02E22D400E0D1
:100FA000302E0FEF502E00E0702E00EC402E0FEF91
:100FB000602E00EC802E00E0902E0FEFB02E00E0AF
:100FC000D02E00E8A02E0FEBC02E00E8E02E09D4B2
:100FD00000E0302E502E702E00EC402E602E802E21
:100FE00000E0902EB02ED02E00E8A02E00ECC02EF7
:100FF000E02EF7D3089507EF302E08E1502E0FEEC4
:10100000702E07EF402E08ED602E0FEE802E0FEDB4
:10101000902E00E6B02E0FEBD02E0FE9A02E00EEA2
:10102000C02E0FEFE02EDDD30FEE302E01E1502E5B
:101030000EEF702E0FEE402E01ED602E0EEF802E83
:101040000FEB902E04E4B02E0BEFD02E0FEBA02E62
:1010500004ECC02E0BEFE02EC4D30EEF302E01E2D5
:10106000502E0FED702E0EEF402E01EE602E0FED84
:10107000802E0BEF902E04E8B02E0FE7D02E0BEB56
:10108000A02E04ECC02E0FEFE02EABD30FED302ED0
:1010900002E2502E0DEF702E0FED402E02EE602E6C
:1010A0000DEF802E0FE7902E08E8B02E07EFD02E20
:1010B0000FEBA02E08ECC02E07EFE02E92D30DEF21
:1010C000302E02E4502E0FEB702E0DEF402E02EC6E
:1010D000602E0FEF802E07EF902E09E0B02E0EEF5E
:1010E000D02E07EBA02E09ECC02E0EEFE02E79D308
:1010F0000FEB302E04E4502E0BEF702E0FEF402E2E
:1011000004EC602E0BEF802E0EEF902E01E1B02E3E
:101110000FEED02E0EEBA02E01EDC02E0FEEE02E26
:1011200060D30BEF302E04E8502E0FE7702E0BEF3C
:10113000402E04EC602E0FEF802E0FEE902E02E179
:10114000B02E0DEFD02E0FEAA02E02EDC02E0DEF27
:10115000E02E47D30FE7302E08E8502E07EF702E11
:101160000FEF402E08EC602E07EF802E0DEF902E33
:1011700002E2B02E0FEDD02E0DEBA02E02EEC02E0F
:101180000FEDE02E2ED308950FEF302E0FE0502EEE
:1011900000EF702E0FEF402E00EC602E0FEF802E30
:1011A000902E00E0B02E0FEFD02E03E8A02E0CEF13
:1011B000C02E0FEFE02E15D300EF302E0FEF502E84
:1011C0000FE0702E0FEF402E00EC602E0FEF802E00
:1011D000902E00E0B02E0FEFD02E0FEBA02E00ECE3
:1011E000C02E0FEFE02EFDD20FE0302E00EF502E7C
:1011F0000FEF702E402E0FEC602E00EF802E0FEFC1
:10120000902E00E0B02E0FEFD02E0FEBA02E00ECB2
:10121000C02E0FEFE02EE5D20FEF302E00E0502E63
:101220000FEF702E00EF402E0FEF602E0FEC802E90
:101230000FEF902E03E0B02E0CEFD02E0FEBA02E70
:1012400000ECC02E0FEFE02ECCD20FEF302E00E0DE
:10125000502E0FEF702E0FEC402E00EF602E0FEF90
:10126000802E0CEF902E0FE3B02E03ECD02E0FEB60
:10127000A02E00ECC02E0FEFE02EB3D20FEF302ED9
:1012800000E0502E0FEF702E402E00EC602E0FEF7E
:10129000802E03EC902E0CEFB02E0FE3D02E0FEB30
:1012A000A02E03ECC02E0CEFE02E9BD20FEF302EC1
:1012B00000E0502E0FEF702E402E00EC602E0FEF4E
:1012C000802E0FE3902E00ECB02E0FEFD02E0CEB03
:1012D000A02E0FEFC02E03ECE02E83D208950EEF68
:1012E000302E0FEF402E03E0502E00EC602E0DEF5D
:1012F000702E0FEF802E902E0FEBA02E00E0B02E60
:1013000000ECC02E0FEFD02EE02E6BD20DEF302E62
:101310000FEF402E06E0502E00EC602E0BEF702EEB
:101320000FEF802E902E0FEBA02E00E0B02E00ECE1
:10133000C02E0FEFD02EE02E54D20BEF302E0FEF39
:10134000402E0CE0502E00EC602E07EF702E0FEFB9
:10135000802E902E0FEBA02E00E0B02E00ECC02EC1
:101360000FEFD02EE02E3DD207EF302E0FEF402EA4
:1013700008E1502E00EC602E0FEE702E0FEF802E45
:10138000902E0FEBA02E00E0B02E00ECC02E0FEF41
:10139000D02EE02E26D20FEE302E0FEF402E00E39F
:1013A000502E00EC602E0FED702E0FEF802E902E41
:1013B0000FEBA02E00E0B02E00ECC02E0FEFD02ED1
:1013C000E02E0FD20FED302E0FEF402E00E6502E04
:1013D00000EC602E0FEB702E0FEF802E902E0FEB97
:1013E000A02E00E0B02E00ECC02E0FEFD02EE02E8D
:1013F000F8D10FEB302E0FEF402E00EC502E602E68
:101400000FE7702E0FEF802E902E0FEBA02E00E036
:10141000B02E00ECC02E0FEFD02EE02EE2D10FE761
:10142000302E0FEF402E00E8502E01EC602E0FEF13
:10143000702E0EEF802E0FEF902E0FEBA02E00E0FF
:10144000B02E00ECC02E0FEFD02EE02ECAD10FEF41
:10145000302E0EEF402E00E0502E03EC602E0FEFEA
:10146000702E0DEF802E0FEF902E0FEBA02E00E0D0
:10147000B02E00ECC02E0FEFD02EE02EB2D10FEF29
:10148000302E0DEF402E00E0502E06EC602E0FEFB8
:10149000702E0BEF802E0FEF902E0FEBA02E00E0A2
:1014A000B02E00ECC02E0FEFD02EE02E9AD10FEF11
:1014B000302E0BEF402E00E0502E0CEC602E0FEF84
:1014C000702E07EF802E0FEF902E0FEBA02E00E076
:1014D000B02E00ECC02E0FEFD02EE02E82D10FEFF9
:1014E000302E07EF402E00E0502E08ED602E0FEF5B
:1014F000702E0FEE802E0FEF902E0FEBA02E00E03F
:10150000B02E00ECC02E0FEFD02EE02E6AD10FEFE0
:10151000302E0FEE402E00E0502E00EF602E0FEF29
:10152000702E0FED802E0FEF902E0FEBA02E00E00F
:10153000B02E00ECC02E0FEFD02EE02E52D10FEFC8
:10154000302E0FED402E00E0502E00EE602E0FEFFB
:10155000702E802E902E0FEBA02E01E0B02E00EC0E
:10156000C02E0EEFD02E0FEFE02E3BD10FEF302E1E
:10157000402E00E0502E00EC602E0FEF702E802EDB
:101580000EEF902E0FEBA02E03E0B02E00ECC02E3D
:101590000DEFD02E0FEFE02E24D10FEF302E402E86
:1015A00000E0502E00EC602E0FEF702E802E0DEF1D
:1015B000902E0FEBA02E06E0B02E00ECC02E0BEF0D
:1015C000D02E0FEFE02E0DD10FEF302E402E00E089
:1015D000502E00EC602E0FEF702E802E0BEF902E11
:1015E0000FEBA02E0CE0B02E00ECC02E07EFD02E9B
:1015F0000FEFE02EF6D00FEF302E402E00E0502EF1
:1016000000EC602E0FEF702E802E07EF902E0FEB68
:10161000A02E08E1B02E00ECC02E0FEED02E0FEF62
:10162000E02EDFD00FEF302E402E00E0502E00ECE9
:10163000602E0FEF702E802E0FEE902E0FEBA02E4F
:1016400000E3B02E00ECC02E0FEDD02E0FEFE02EF9
:10165000C8D00FEF302E402E00E0502E00EC602E50
:101660000FEF702E802E0FED902E0FEBA02E00E6C8
:10167000B02E00ECC02E0FEBD02E0FEFE02EB1D02D
:101680000FEF302E402E00E0502E00EC602E0FEFBA
:10169000702E802E0FEB902EA02E00ECB02EC02EC0
:1016A0000FE7D02E0FEFE02E9CD00FEF302E402E04
:1016B00000E0502E00EC602E0FEF702E802E0FE712
:1016C000902E0FEBA02E00E8B02E01ECC02E0FEFF5
:1016D000D02E0EEFE02E85D00FEF302E402E00E002
:1016E000502E00EC602E0FEF702E802E902E0EEB01
:1016F000A02E00E0B02E03ECC02E0FEFD02E0DEF89
:10170000E02E6FD00FEF302E402E00E0502E00EC78
:10171000602E0FEF702E802E902E0DEBA02E00E08D
:10172000B02E06ECC02E0FEFD02E0BEFE02E59D0CE
:101730000FEF302E402E00E0502E00EC602E0FEF09
:10174000702E802E902E0BEBA02E00E0B02E0CEC15
:10175000C02E0FEFD02E07EFE02E43D00FEF302E2C
:10176000402E00E0502E00EC602E0FEF702E802EE9
:10177000902E07EBA02E00E0B02E08EDC02E0FEF4C
:10178000D02E0FEEE02E2DD00FEF302E402E00E0A9
:10179000502E00EC602E0FEF702E802E902E0FEA50
:1017A000A02E00E0B02E00EFC02E0FEFD02E0FEDD8
:1017B000E02E17D00FEF302E402E01E0502E00EC1F
:1017C000602E0EEF702E0FEF802E902E0FE9A02EC0
:1017D00000E0B02E00EEC02E0FEFD02EE02E01D094
:1017E000089544D343D3889588958895889588959E
:1017F0008895C0D308950FEF302E00E0502E0FEFE4
:10180000702E402E00EC602E0FEF802E902E00E008
:10181000B02E0FEFD02E0FEBA02E00ECC02E0FEF4E
:10182000E02EDFDF0EEF302E0FEF402E902E09E975
:10183000A02E01E0502E00EC602E00E0B02E0CEC4B
:10184000C02E0FEF702E802ED02E01EEE02EC9DFBD
:101850000CEF302E0FEF402E902E03EBA02E02E067
:10186000502E00EC602E00E0B02E08EDC02E0FEFE1
:10187000702E802ED02E03ECE02EB3DF09EF302E39
:101880000FEF402E902E07EAA02E04E0502E00EC21
:10189000602E00E0B02E00EFC02E0EEF702E0FEF86
:1018A000802ED02E07ECE02E9CDF03EF302E0FEFC2
:1018B000402E902E0FE8A02E09E0502E00EC602E56
:1018C00000E0B02E00EEC02E0CEF702E0FEF802E39
:1018D000D02E0FECE02E85DF06EE302E0FEF402EDF
:1018E000902E0FE9A02E03E1502E00EC602E00E0B8
:1018F000B02E00ECC02E08EF702E0FEF802ED02EF1
:101900000FEDE02E6EDF0CEC302E0FEF402E902E00
:101910000FEBA02E06E2502E00EC602E00E0B02E61
:1019200000ECC02E00EF702E0FEF802ED02EE02E98
:1019300058DF09E9302E0FEF402E902E0FEBA02E2E
:101940000CE4502E00EC602E00E0B02E00ECC02E17
:1019500001EE702E0FEF802ED02EE02E42DF03E33B
:10196000302E0FEF402E902E0FEBA02E08E9502EB8
:1019700000EC602E00E0B02E00ECC02E03EC702EC8
:101980000FEF802ED02EE02E2CDF07E6302E0EEF4C
:10199000402E0FEF902E0FEBA02E00E3502E01EC07
:1019A000602E00E0B02E00ECC02E07E8702E0FEF86
:1019B000802ED02EE02E15DF0FEC302E0CEF402EB7
:1019C0000FEF902E0FEBA02E00E6502E02EC602EB3
:1019D00000E0B02E00ECC02E0FE0702E0FEF802E36
:1019E000D02EE02EFEDE0FE9302E09EF402E0FEF55
:1019F000902E0FEBA02E00EC502E04EC602E00E099
:101A0000B02E00ECC02E0FE1702E0EEF802E0FEFE7
:101A1000D02EE02EE6DE0FE3302E03EF402E0FEF48
:101A2000902E0FEBA02E00E8502E09EC602E00E067
:101A3000B02E00ECC02E0FE3702E0CEF802E0FEFB7
:101A4000D02EE02ECEDE0FE7302E06EE402E0FEF2A
:101A5000902E0FEBA02E00E0502E03ED602E00E044
:101A6000B02E00ECC02E0FE7702E08EF802E0FEF87
:101A7000D02EE02EB6DE0FEF302E0CEC402E0FEF06
:101A8000902E0FEBA02E00E0502E06EE602E00E010
:101A9000B02E00ECC02E0FEF702E00EF802E0FEF57
:101AA000D02EE02E9EDE0FEF302E09ED402E0EEFF1
:101AB000902E0FEBA02E00E0502E0CEC602E01E0DB
:101AC000B02E00ECC02E0FEF702E01EE802E0FEF27
:101AD000D02EE02E86DE0FEF302E03EF402E0CEFDF
:101AE000902E0FEBA02E00E0502E08ED602E02E0AD
:101AF000B02E00ECC02E0FEF702E03EC802E0FEFF7
:101B0000D02EE02E6EDE0FEF302E07EE402E09EFC6
:101B1000902E0FEBA02E00E0502E00EF602E04E080
:101B2000B02E00ECC02E0FEF702E07EC802E0EEFC3
:101B3000D02E0FEFE02E55DE0FEF302E0FEC402EA3
:101B400003EF902E0FEBA02E00E0502E00EE602E43
:101B500009E0B02E00ECC02E0FEF702E0FEC802E9F
:101B60000CEFD02E0FEFE02E3CDE0FEF302E0FEDFE
:101B7000402E06EE902E0FEBA02E00E0502E00EC33
:101B8000602E03E1B02E00ECC02E0FEF702E0FED93
:101B9000802E08EFD02E0FEFE02E23DE0FEF302E39
:101BA000402E0CEC902E0FEBA02E00E0502E00ECFF
:101BB000602E06E2B02E00ECC02E0FEF702E802EAD
:101BC00000EFD02E0FEFE02E0CDE0FEF302E402E68
:101BD00009E9902E0FEBA02E00E0502E00EC602EB5
:101BE0000CE4B02E00ECC02E0FEF702E802E01EE14
:101BF000D02E0FEFE02EF5DD0FEF302E402E03E359
:101C0000902E0FEBA02E00E0502E00EC602E08E985
:101C1000B02E00ECC02E0FEF702E802E03ECD02ED5
:101C20000FEFE02EDEDD0FEF302E402E07E6902E78
:101C30000EEBA02E00E0502E00EC602E00E3B02E44
:101C400001ECC02E0FEF702E802E07E8D02E0FEF84
:101C5000E02EC7DD0FEF302E402E0FEC902E0CEB58
:101C6000A02E00E0502E00EC602E00E6B02E02EC1C
:101C7000C02E0FEF702E802E0FE0D02E0FEFE02E33
:101C8000B0DD0FEF302E402E0FE9902E09EBA02E85
:101C900000E0502E00EC602EB02E04ECC02E0FEFB2
:101CA000702E802E0FE1D02E0EEFE02E9ADD0FEF7A
:101CB000302E402E0FE3902E03EBA02E00E0502E8E
:101CC00000EC602E00E8B02E09ECC02E0FEF702E55
:101CD000802E0FE3D02E0CEFE02E83DD0FEF302EA1
:101CE000402E0FE7902E06EAA02E00E0502E00ECCA
:101CF000602E00E0B02E03EDC02E0FEF702E802E70
:101D00000FE7D02E08EFE02E6CDD0FEF302E402EC7
:101D1000902E0CE8A02E00E0502E00EC602E00E08B
:101D2000B02E06EEC02E0FEF702E802ED02E00EFBC
:101D3000E02E57DD089517FC02C000E8102A089530
:101D400000FE02C00EEF102201FE02C00DEF1022B5
:101D500002FE02C00BEF102203FE02C007EF1022AA
:101D600004FE02C00FEE102205FE02C00FED10228D
:101D700006FE02C00FEB102207FE02C00FE7102282
:101D800008950F921F920FB70F93FF920F93B79979
:101D900003C001E00093600015E0211608F046C082
:101DA00014E02116C1F113E0211651F112E02116C1
:101DB000E1F011E0211671F010E0211601F0AD986C
:101DC000032C1FEF012602BA042C1FE3012608BAD8
:101DD000A89A39C0A898052C1FEF012602BA062C34
:101DE0001FE3012608BAA99A2EC0A998072C1FEF55
:101DF000012602BA082C1FE3012608BAAA9A23C0BA
:101E0000AA98092C1FEF012602BA0A2C1FE7012607
:101E100008BAAB9A18C0AB980B2C1FEF012602BA78
:101E20000C2C1FE7012608BAAC9A0DC000E0202E4A
:101E3000AC980D2C1FEF012602BA0E2C1FE70126CD
:101E400008BAAD9A01C023940F91FF900F910FBF74
:101E50001F900F9018950AD009D008D007D006D04F
:101E600005D004D003D002D001D008950AD009D003
:101E700008D007D006D005D004D003D002D001D0BE
:101E8000089505D004D003D002D001D008958895DC
:101E9000089500916000003051F0B79B08C0009198
:101EA000610003950093610000E0009360000091E1
:101EB0006100003009F41AD600916100013009F484
:101EC0000EDA00916100023009F426D6009161001B
:101ED000033009F46FD400916100043009F48BD809
:101EE00000916100053009F45CD300916100063077
:101EF00009F44AD900916100073009F46FD20091CA
:101F00006100083009F414D700916100093009F428
:101F10005CD1009161000A3009F4D3D700916100CF
:101F20000B3009F480D0009161000C3009F47ADCA8
:101F3000009161000D3009F41FD5009161000E3051
:101F400009F470D5009161000F3009F489D4009133
:101F50006100003109F485D600916100013109F476
:101F600019D600916100023108F493CF00E000938C
:101F700061009DCF00916000003019F0B79B01C057
:041F800088DF089559
:00000001FF
